:020000040000FA
:020000005D2879
:08000800A22B2208A10208004E
:100010002208A1070800A20908002208A10608007A
:10002000A30121082218A3070310A20C0310A10D9D
:10003000A208031D112808002208A1050800A80134
:10004000A901261830200310A70CA60C0310A40D3C
:10005000A50DA608031D2128A708031D21280800B7
:100060002408A8070318A90A2508A90708002108D9
:10007000A202031D003401342108A202031C003433
:100080000134B00908003008AF0708002F08B0029B
:10009000031D003401343208B4023308031C330F4B
:1000A000B502031C003401343208B402031D0034CD
:1000B0003308B502031D0034013483120313850194
:1000C00007309F008316031300308500831203134B
:1000D0008601831603130030860083120313DA307F
:1000E000AC008830AA009A30AB00AB0B7528AA0B85
:1000F0007328AC0B71280000000000000000000015
:1001000000000000000000000000000000000000EF
:1001100000000000000000000000000000000000DF
:1001200000000000000000000000000000000000CF
:100130000000000000000000831603138617060865
:1001400070388600073083120313C5004508A100EC
:100150009523831203132008A200052083120313A2
:100160002108C500861FC728831203134508C20053
:100170000F30C3004208A1000030A20037208312D4
:100180000313A3002318C528C6281B23CD2800303D
:1001900083120313C2004508C300FA30831203130D
:1001A000C0000030C1004208C4000723E8308312B9
:1001B0000313C0000330C100DE2219308312031381
:1001C000C0000030C1001430C4000723E83083129F
:1001D0000313C0000330C100DE2291018316031314
:1001E00078309200831203133C30950097010F3052
:1001F0009704203097048316031386118312031388
:10020000121500309204831603138C10831203130B
:1002100012118316031386140615773099001811EE
:100220001812831203139817181318168316031342
:10023000181398161817A03083120313CD0000303E
:10024000CE0083134E188317831203134D088400C6
:1002500055308000CD0A0319CE0A8313831203138D
:100260004E188317831203134D088400FF3080005B
:10027000CD0A0319CE0A8313831203134E18831772
:10028000831203134D08840000308000CD0A031947
:10029000CE0A8313831203134E188317831203139A
:1002A0004D088400F7308000CD0A0319CE0A83136D
:1002B000831203134E188317831203134D0884000F
:1002C00008308000CD0A0319CE0AA0308312031330
:1002D000D8000030D900AB30D5000030D600003057
:1002E000D40018178C12831603138C168B170B1758
:1002F0008312031385140511E830DC000330DD00A0
:10030000DC0A0319DD0A83120313DC080319DD0379
:1003100083120313DC03DD08031D912983120313E9
:10032000DC080319C229831203130508A100063053
:10033000A2000D2083120313210885003B30AC007E
:100340000530AA000530AB00AB0BA429AA0BA229EB
:10035000AC0BA029831203130508A1000630A200EC
:100360000D2083120313210885003B30AC000530BB
:10037000AA000530AB00AB0BBB29AA0BB929AC0B0B
:10038000B7298329831203134208A1000030A20079
:10039000372083120313A3002318D32900308312BC
:1003A0000313BF00D729023083120313BF00831247
:1003B00003133F08A1000230A20037208312031369
:1003C000A3002318E429462A831203134208C90014
:1003D0004208A1000030A200372083120313A300BB
:1003E0002318F729003083120313BF000F2A83124A
:1003F00003134308BE003E08A1001030A2001020E5
:10040000831203132308BE004908A1003E08A2007E
:100410000820831203132108C9000130BF002623DE
:10042000323083120313CA00CA0A83120313CA03A9
:1004300003193D2A831203130508A1000630A20008
:100440000D2083120313210885000B30AC00AC0B88
:10045000272A00000000831203130508A1000630BC
:10046000A2000D2083120313210885000B30AC007D
:10047000AC0B382A00000000152A14308312031335
:10048000C0000030C1000530C400072383120313ED
:100490003F08A1000030A200372083120313A300FD
:1004A0002318532A7D2A831203134B08A10001301D
:1004B000A200372083120313A3002318602A7D2A89
:1004C000831203134608A1000F30A2001C208312E0
:1004D00003132108C6004608A1000030A2003720FF
:1004E00083120313A3002318762A7A2A0130831279
:1004F0000313BF0083120313CB01831203133F08BE
:10050000A1000130A200372083120313A300231897
:100510008A2ABA2A831203134208A1000030A200DB
:10052000372083120313A30023189C2A831203137A
:100530004208C000C101A42A831203134308C0006B
:10054000C101C00A0319C10A831203134008A400A1
:100550004108A500E830A6000330A7001F20831241
:1005600003132808C0002908C100DE2202308312CC
:100570000313BF00831203133F08A1000230A2003F
:100580003C2083120313A3002318DC2A83120313D5
:100590004208A1000030A200372083120313A300F9
:1005A0002318D72A003083120313BF00DB2A02303E
:1005B00083120313BF00DC2AD729DD2A8312031319
:1005C0004008C7004108C800C70A0319C80A8312B7
:1005D0000313C7080319C80383120313C703C8080A
:1005E000031DF52A83120313C7080319062B831270
:1005F00003133B30AC000530AA000530AB00AB0B59
:10060000FF2AAA0BFD2AAC0BFB2AE72A080083125B
:1006100003134408CC00CC0A83120313CC03031940
:100620001A2B831203130514DE2283120313051001
:10063000DE220C2B0800203083120313C000003090
:10064000C1000130C4000723232B0800A53083120A
:100650000313CD000030CE0083134E18831783128E
:1006600003134D08840049088000CD0A0319CE0AFF
:10067000F73083120313D0005008A1004908A200EC
:100680000820831203132108D0004908A2000B2080
:10069000831203132208CF0083134E18831783128B
:1006A00003134D0884004F088000CD0A0319CE0AB9
:1006B0008313831203134E188317831203134D08F9
:1006C000840050088000CD0A0319CE0A8312031358
:1006D0005008A2000B20831203132208CF008313BB
:1006E0004E188317831203134D0884004F088000AF
:1006F000A030CD000030CE0012150C12831603136B
:100700000C168B170B170800A03083120313D800A8
:100710000030D900AB30D5000030D6000030D40016
:100720001A08D7001A08DA00080083120313A00180
:100730002010061A2014A010861AA0142011061BDF
:1007400020150800FF00030E83120313BC007F086E
:10075000BD002008AE00831603130C1EB72B8312B6
:1007600003130C1EB72BCE23831203130C12831614
:1007700003138C1EC32B831203138C1EC32B2D2437
:10078000831203138C12831203132E08A0003D085A
:10079000FF003C0E8300FF0E7F0E090083138312BF
:1007A00003134E188317831203134D0884000008A7
:1007B000C5004508D200D1010830D300D30A831206
:1007C0000313D3030319F72B83120313521CE92BD2
:1007D000F22B831203135108B0004120831203133C
:1007E0003008D100031083120313D20CDF2B8312C5
:1007F00003135108AF000030B000462083120313EA
:10080000B1003118072C8316031318100A2C831615
:1008100003131814831203130C1E0C2C83120313DE
:1008200045089900CD0A0319CE0A831203134D0817
:10083000B2004E08B300AA30B4000030B5004B201F
:1008400083120313B10031182C2C831603130C12DE
:100850008312031312112C2C080083120313981C0B
:10086000332C18121816831203131A08DB00831393
:100870005618831783120313550884005B08800001
:100880005508B2005608B300AE30B4000030B500D1
:10089000542083120313B10031184F2C532C8312B0
:1008A00003135B08D400831203135508B2005608E3
:1008B000B300AF30B4000030B5004B2083120313F7
:1008C000B1003118642C792C831203135B08AF003C
:1008D00083135918831783120313580884000008E0
:1008E000B000462083120313B1003118792C842301
:1008F000792C831203135508B2005608B300B030A8
:10090000B4000030B500542083120313B100311835
:100910008A2C9E2C831203135B08D7005B08B0005F
:100920004120831203133008DA005408AF005B083B
:10093000B0004320831203132F08D4008312031343
:100940005508B2005608B300B130B4000030B5000D
:10095000542083120313B1003118AF2CBD2C831225
:1009600003135B08AF005A08B0004620831203133C
:10097000B1003118BD2C8423BD2C831203135508FC
:10098000B2005608B300B230B4000030B5005420B5
:1009900083120313B1003118CE2CE52C83120313FC
:1009A0005B08AF005408B000462083120313B10067
:1009B0003118DC2C8423DC2C831203135B08B00079
:1009C0004120831203133008DA0083120313550801
:1009D000B2005608B300B330B4000030B500542064
:1009E00083120313B1003118002D83120313D80AA8
:1009F0000319D90A83120313D50A0319D60A212D24
:100A0000831203135B08AF005A08B000462083121C
:100A10000313B10031180D2D202D831203134B0841
:100A2000AF000130B000462083120313B10031182B
:100A3000202D013083120313CB005708C600202D50
:040A40008423080003
:02400E00023F6F
:00000001FF
